:020000040000FA
:100000000C94F3010C94770B0C94500B0C941B0282
:100010000C941B020C941B020C941B020C941B02EC
:100020000C941B020C941B020C941B020C941B02DC
:100030000C941B020C941B020C941B020C941B02CC
:100040000C94060B0C941B020C941B020C941B02C8
:100050000C941B020C941B020C941B020C941B02AC
:100060000C949E0B0C941B02000038387C7CFEFE26
:10007000FEFFFEFFFC7FF83FF01FE00FC00780038C
:10008000000100000000000053704F323A00424D62
:10009000503A004F464620494E0074616E746169C3
:1000A0007A696E696E67004D6164652062790052FD
:1000B00061770041766700495200526564004469E7
:1000C00073706C61790046494E47455200504C416F
:1000D000434500446576696365206572726F7200FE
:1000E000A81FD30040A1C8DA0281FFA4A6D5808D45
:1000F00014AF00000000240027002A0000000000C8
:10010000250028002B005F5F5F60606061616161B6
:1001100061626262626263636363636363636464B4
:10012000646464646464646464646464646464648F
:100130006464636363636363636362626262626293
:1001400061616161606060605F5F5F5E5E5E5D5DBA
:100150005D5C5C5C5B5B5A5A595959585857575605
:100160005655555454535252515150504F4E4E4D76
:100170004C4C4B4A4A49484847464545444342420D
:1001800041403F3E3E3D3C3B3A39383837363534C6
:10019000333231302F2E2D2C2B2A292827262524A7
:1001A0002322211F1E1D1C1B1A19171615141311AB
:1001B000100F0E0C0B0A09070605030201000000D0
:1001C000000023002600290004040404040404049D
:1001D00002020202020203030303030301020408F2
:1001E00010204080010204081020010204081020A1
:1001F00000000008000201000003040700000000E6
:1002000000000000000000000000005F0000000788
:10021000000700147F147F14242A7F2A1223130856
:10022000646236495620500008070300001C224132
:10023000000041221C002A1C7F1C2A08083E0808D6
:100240000080703000080808080800006060002086
:10025000100804023E5149453E00427F4000724969
:100260004949462141494D331814127F102745450D
:1002700045393C4A49493141211109073649494923
:1002800036464949291E0000140000004034000091
:1002900000081422411414141414004122140802FA
:1002A000015909063E415D594E7C1211127C7F496D
:1002B0004949363E414141227F4141413E7F4949C2
:1002C00049417F090909013E414151737F080808EE
:1002D0007F00417F41002040413F017F08142241BF
:1002E0007F404040407F021C027F7F0408107F3E19
:1002F0004141413E7F090909063E4151215E7F0986
:10030000192946264949493203017F01033F4040EC
:10031000403F1F2040201F3F4038403F63140814D7
:100320006303047804036159494D43007F4141410F
:100330000204081020004141417F040201020440F0
:1003400040404040000307080020545478407F2874
:100350004444383844444428384444287F3854546A
:10036000541800087E090218A4A49C787F0804048D
:100370007800447D40002040403D007F102844002C
:1003800000417F40007C047804787C0804047838BD
:1003900044444438FC1824241818242418FC7C08ED
:1003A000040408485454542404043F44243C40406A
:1003B000207C1C2040201C3C4030403C442810281D
:1003C000444C9090907C4464544C44000836410066
:1003D000000077000000413608000006090600FF13
:1003E000FFFFFFFFBD0C11241FBECFEFD8E0DEBF23
:1003F000CDBF11E0A0E0B1E0E6E7F3E202C0059076
:100400000D92A631B107D9F723E0A6E1B1E001C012
:100410001D92AD35B207E1F711E0C3EFD1E004C0A2
:100420002197FE010E94A411C23FD107C9F70E9483
:10043000F60C0C94B9110C940000262F26952695E5
:1004400026959091DC0229130EC0E82FF0E0E452CB
:10045000FD4F677021E030E001C0220F6A95EAF796
:100460008181822B818308952F923F924F925F92D8
:100470006F927F928F929F92AF92BF92CF92DF92B4
:10048000EF92FF920F931F93CF93DF93562E790134
:100490004052550B95E0949F9001959F300D11248B
:1004A000570153E0AA0CBB1C5A95E1F76E2C782E2D
:1004B00010E000E0C9018C5F9D4F6C01882483949B
:1004C000912CF601E00FF11FE491CE2FD0E092E0E5
:1004D000E916F104F9F484E0CC0FDD1F8A95E1F709
:1004E000CC27DF70EF70CE018E2BEC01CC0FDD1F1F
:1004F000CC0FDD1F8C2B9D2B83739373EC01CC0FE2
:10050000DD1FC82BD92BC575D575CE01880F991F56
:10051000C82BD92B312C3E141F04D4F4232C270CC8
:10052000412C4A141B0494F4C401042C02C0880F0B
:10053000991F0A94E2F78C239D23892B29F0642DBF
:10054000650D822D0E941D024394EBCF3394E3CFBF
:100550000F5F1F4F760C0530110509F0B2CFDF9108
:10056000CF911F910F91FF90EF90DF90CF90BF90B0
:10057000AF909F908F907F906F905F904F903F9043
:100580002F9008953F924F925F926F927F928F9239
:100590009F92AF92BF92CF92DF92EF92FF920F9312
:1005A0001F93CF93DF935B0169017A012AEF200348
:1005B0004001219F900C11242CE0209FE001219FFD
:1005C000D00D1124C80FD91F83E0382E9AE0492E90
:1005D000512C612C712C40E2C114D104E104F104CE
:1005E00041F0C701B601A30192010E94501140E3FE
:1005F000460F9801B501CE010E943402C701B60131
:10060000A30192010E94501169017A013A94C80D28
:10061000D91D3110E0CFDF91CF911F910F91FF9045
:10062000EF90DF90CF90BF90AF909F908F907F9092
:100630006F905F904F903F900895EF92FF920F93CD
:100640001F93CF93DF938C017B012091DC02862FD7
:100650008695869586952817D0F0CB01079633E0CE
:10066000959587953A95E1F72817190609F07CF4D6
:10067000EA01FE0144912196442349F021E030E053
:10068000B701C8010E9434020A5F1F4FF2CFDF9109
:10069000CF911F910F91FF90EF900895833081F0DB
:1006A00028F4813099F08230A9F008958730A9F0BC
:1006B0008830C9F08430B1F4809180008F7D03C010
:1006C000809180008F7780938000089584B58F7724
:1006D00084BD089584B58F7DFBCF8091B0008F7766
:1006E0008093B00008958091B0008F7DF9CFCF93B3
:1006F000DF93E3EFF1E08491EFEDF1E0D491EBECE7
:10070000F1E0C491CC23A1F081110E944E03EC2FA3
:10071000F0E0EE0FFF1FE254FE4FA591B491EC9173
:10072000ED2381E090E009F480E0DF91CF9108951E
:1007300080E090E0FACF1F93CF93DF93282F30E033
:10074000F901E051FE4F8491F901E452FE4FD4913A
:10075000F901E853FE4FC491CC23A9F0162F811163
:100760000E944E03EC2FF0E0EE0FFF1FE450FF4F0E
:10077000A591B4918FB7F894EC91111108C0D09560
:10078000DE23DC938FBFDF91CF911F910895DE2B85
:10079000F8CFCF93DF9390E0FC01E452FE4F249119
:1007A00088539E4FFC0184918823C9F090E0880F04
:1007B000991FFC01EE50FF4FA591B491FC01E4504C
:1007C000FF4FC591D49161110DC09FB7F8948C91E2
:1007D000209582238C938881282328839FBFDF91D3
:1007E000CF910895623051F49FB7F8943C91822FD5
:1007F000809583238C93E8812E2BEFCF8FB7F894CD
:10080000EC912E2B2C938FBFEACF3FB7F8948091B9
:100810005F0190916001A0916101B091620126B5E4
:10082000A89B05C02F3F19F00196A11DB11D3FBF28
:10083000BA2FA92F982F8827BC01CD01620F711DF7
:10084000811D911D42E0660F771F881F991F4A95F1
:10085000D1F708958F929F92AF92BF92CF92DF927D
:10086000EF92FF924B015C010E9405046B017C0139
:100870000E9405046C197D098E099F09683E73402A
:1008800081059105A8F321E0821A9108A108B10819
:1008900088EEC80E83E0D81EE11CF11C811491047F
:1008A000A104B10429F7FF90EF90DF90CF90BF90A3
:1008B000AF909F908F900895089520913901260F51
:1008C0003327331F21323105ECF42091C501FC019F
:1008D00090E080E0243069F082E00895A091390131
:1008E0002191AC01495E5E4FA40FB52FB11D2C9331
:1008F0000196861798F380913901680F609339014A
:1009000080E0089581E008951092C50181E0809310
:10091000C40110929F0161E082E10E949B0361E0AB
:1009200083E10E949B03E9EBF0E080818E7F80836E
:1009300080818D7F808388E48093B80085E48093F4
:10094000BC000895CF93DF9391E090931601882324
:10095000B9F0C091B800D091BA008091BC008A7BF8
:100960008093BC0060E082E10E949B0360E083E131
:100970000E949B030E948404D093BA00C093B800E5
:10098000DF91CF910895CF92DF92EF92FF920F9374
:100990001F93CF93DF93D091EE0181E0D13208F025
:1009A0009CC0C091ED010E9405046B017C01809107
:1009B000C50181116CC082E08093C50181E0809304
:1009C000C4018FEF8093C3011092C201D093C10183
:1009D000ADECB1E0E1EAF1E080E0D8138DC0109217
:1009E000A0018091A001CC0FC82BC093A0018091E1
:1009F0009F01813009F084C010929F010E9405047C
:100A00006B017C018091A0018093BB008091C701A4
:100A10009091C801A091C901B091CA01892B8A2B7C
:100A20008B2BA1F00E9405040091C7011091C80111
:100A30002091C9013091CA016C197D098E099F0965
:100A4000061717072807390708F442C08091BC0031
:100A500083FDD8CF85EC8093BC000E9405046B0118
:100A60007C018091C501823009F44CC08091C301A2
:100A70008F3F09F469C08091C301803209F466C0D8
:100A80008091C301803309F463C084E026C0809163
:100A9000C7019091C801A091C901B091CA01892BE9
:100AA0008A2B8B2B09F483CF0E9405040091C70188
:100AB0001091C8012091C9013091CA016C197D09BA
:100AC0008E099F09061717072807390708F06FCF07
:100AD0008091C6010E94A20485E01092CC01109280
:100AE000EE011092CB01DF91CF911F910F91FF90FA
:100AF000EF90DF90CF9008959D9191938F5F6DCF90
:100B000085EEA9CF8091C7019091C801A091C9013C
:100B1000B091CA01892B8A2B8B2B09F4A2CF0E949A
:100B200005040091C7011091C8012091C9013091BD
:100B3000CA016C197D098E099F0906171707280736
:100B4000390708F08ECFC4CF80E0C7CF82E0C5CF91
:100B500083E0C3CFCF92DF92EF92FF920F931F9368
:100B6000CF93DF93D82FC62F613208F098C00E9430
:100B700005046B017C018091C50181116BC081E08E
:100B80008093C5018093C4019FEF9093C30110929D
:100B9000C2019C0F9093C1018093A0018091A0019C
:100BA000DD0FD82BD093A00180919F01813009F0F7
:100BB00078C010929F010E9405046B017C01809116
:100BC000A0018093BB008091C7019091C801A091C2
:100BD000C901B091CA01892B8A2B8B2BA1F00E94ED
:100BE00005040091C7011091C8012091C9013091FD
:100BF000CA016C197D098E099F0906171707280776
:100C0000390708F448C08091BC0083FDD8CF85EC3B
:100C10008093BC000E9405046B017C018091C5019A
:100C2000813009F440C08091C2018C1710F4C0914A
:100C3000C201E1EAF1E0AFE7B1E080E08C1355C01A
:100C40008C2FDF91CF911F910F91FF90EF90DF904C
:100C5000CF9008958091C7019091C801A091C901DA
:100C6000B091CA01892B8A2B8B2B09F484CF0E9467
:100C700005040091C7011091C8012091C90130916C
:100C8000CA016C197D098E099F09061717072807E5
:100C9000390708F070CF8091C6010E94A204C0E01D
:100CA000CFCF85EEB5CF8091C7019091C801A091BB
:100CB000C901B091CA01892B8A2B8B2B09F4AECFC5
:100CC0000E9405040091C7011091C8012091C9013B
:100CD0003091CA016C197D098E099F090617170703
:100CE0002807390708F09ACFD6CF91919D938F5F4F
:100CF000A5CF089508950895E0917E0180917D012A
:100D0000E81730F4F0E0E158FE4F808190E008955C
:100D10008FEF9FEF089590917E0180917D012FEFDD
:100D20003FEF981748F4E92FF0E0E158FE4F20819B
:100D300030E09F5F90937E01C9010895CF92DF92CA
:100D4000EF92FF92F12C8FEE91E00E948B06E82E3D
:100D50008FEE91E00E948B06D82E8FEE91E00E94DC
:100D60008B06C82EC701B60183709927FF90EF90BC
:100D7000DF90CF90089580917D0190917E01891B35
:100D8000990B0895CF92DF92EF92FF920F931F93EA
:100D9000CF93DF937C01CB018A012091CB012223E9
:100DA00089F0EB016B01C40ED51ECC15DD0569F091
:100DB0006991D701ED91FC910190F081E02DC7017F
:100DC0000995F3CF642F0E945D04C801DF91CF9194
:100DD0001F910F91FF90EF90DF90CF900895CF93E8
:100DE000DF931F92CDB7DEB769832091CB01222319
:100DF000F9F02091EE01203258F021E030E0FC01C2
:100E00003383228390E080E00F90DF91CF910895AB
:100E10008091CC01E82FF0E0E353FE4F998190835D
:100E20008F5F8093CC018093EE0181E090E0ECCF66
:100E300061E0CE0101960E945D04F7CF682F8FEE2E
:100E400091E00C94EF0681E08093CB018CE38093DA
:100E5000ED011092CC011092EE0180E490E00C9430
:100E60001E0781E08093CB018CE38093ED0110920B
:100E7000CC011092EE0190E080E00C941E07CF931D
:100E8000C62F9091C10221E02093CB019093ED01F8
:100E90001092CC011092EE01682F8FEE91E00E942B
:100EA000EF066C2F8FEE91E00E94EF06CF910C942D
:100EB000C304CF93DF93C82FD62F0E94310780E25F
:100EC00090E00E941E0781E090E00E941E0781E2F0
:100ED00090E00E941E0760E08FEE91E00E94EF0616
:100EE0008FE790E00E941E0782E290E00E941E07BA
:100EF0006C2F8FEE91E00E94EF062C2F2D0F3327E1
:100F0000331FC90101970E941E07DF91CF910C94F6
:100F1000C304CF93DF9364E080E00E9459070E94EE
:100F20002307C0E0D2E060E08FEE91E00E94EF0680
:100F3000892B49F40E94C3040E94230760E08FEECE
:100F400091E00E94EF06219771F7DF91CF910C9409
:100F5000C30490E080E0089581E0809368010895E3
:100F6000FC01208530E0D901AA0FBB1FA80FB91FD3
:100F70006D937C932F5F3F4F237033272087208111
:100F8000318182819381280F391F84819581280FB7
:100F9000391F86819781820F931F97FD0396959540
:100FA0008795959587950895CF93DF93FC01838965
:100FB00044895589882351F14617570734F4708BBB
:100FC000678780E032C080E01DC064177507CCF7EA
:100FD00027853089A189B2892A1B3B0BD9015597F6
:100FE000A33ABB4080F7A585B685ED01B7FD2396F2
:100FF000D595C795D595C7952C1B3D0B2A0F3B1F43
:1010000036872587128A118A138A05C064177507E7
:101010002CF4728B618B9389911107C04617570787
:1010200024F4108A178691E0938B758B648BDF9183
:10103000CF910895CF93DF93C1ECD2E0988121E066
:101040002093CB019093ED011092CC011092EE0110
:10105000682F8FEE91E00E94EF060E94C30461E0CA
:1010600088810E94AA0510927E0180937D018FEEF7
:1010700091E00E948B06C82F0E94C3048C2FDF9141
:10108000CF91089585ED8093BC008091C701909128
:10109000C801A091C901B091CA010796A11DB11D57
:1010A00023E0B695A795979587952A95D1F7209136
:1010B000BC0024FD03C01092C50108954091C701F2
:1010C0005091C8016091C9017091CA01452B462B0E
:1010D000472B69F30097A105B10541F025E32A9557
:1010E000F1F700000197A109B109E1CF8091C60194
:1010F0000C94A2046F927F928F929F92AF92BF92B4
:10110000CF92DF92EF92FF920F931F93CF93DF93D3
:101110007C011092DC025AE0852E64E4762E7DED8F
:10112000A72E72E0B72E83E0E816F10409F490C10F
:101130000CF050C0F1E0EF16F10409F4B8C082E001
:10114000E816F10409F415C143ED50E070E060E0E9
:101150008AE090E00E941D038091DC0291E0980FEC
:101160009093DC0261E00E9459070E9423070DED75
:1011700012E0C0E0F801D1918F016D2F8FEE91E068
:101180000E94EF06892B49F40E94C3040E942307A2
:101190006D2F8FEE91E00E94EF06CF5FC03851F7C0
:1011A0000E94C304F5011192CA95E9F78091DC020F
:1011B000843009F0B8CFDF91CF911F910F91FF904C
:1011C000EF90DF90CF90BF90AF909F908F907F90E7
:1011D0006F900895E4E0EE16F10409F448C1F5E0DB
:1011E000EF16F10409F0B0CF4EE850E070E060E097
:1011F00090E080E00E941D03209172013091730104
:10120000032E000C440B550B02E010E070E060E090
:1012100089E190E00E94C20248E850E06FE070E08F
:1012200090E080E00E941D0320916D0130916E01DD
:10123000032E000C440B550B6FE070E089E190E049
:101240000E94C2028091DC028150823008F084CF7B
:1012500010E000E028E0D22ED0E0C0E0CE018770A0
:101260009927009759F4FE0193E0F595E7959A9533
:10127000E1F7E00FF11FE859FF4F9490292D30E07E
:1012800002C0359527958A95E2F720FF05C06D2DA0
:101290008C2F86590E941D022196C031D105F1F68E
:1012A000D3940E5F1F4FF8E1DF12D6CF55CF4DEC30
:1012B00050E06AE070E08DE090E00E941D0346EC93
:1012C00050E064E170E08AE090E00E941D038091AC
:1012D0007B0190917C016AE070E00E943C11C82F74
:1012E00040E3460F21E030E070E060E084E690E00B
:1012F0000E94340221E030E04EE270E060E08AE6D5
:1013000090E00E94340240E34C0F21E030E070E0B6
:1013100060E080E790E00E94340221E030E046E5A2
:1013200070E060E086E790E00E9434024EEB50E00F
:101330006EE070E084E590E00E941D0380917801EA
:101340004AEB50E0811102C047EB50E068E170E0E9
:1013500084E590E00E941D03809179014FEA50E0FE
:10136000882311F043EB50E068E170E08CE690E0F8
:10137000F1CE2091720130917301032E000C440BC9
:10138000550B02E010E070E060E086E590E00E941E
:10139000C20243E4C42E42E0D42E10E000E0F60185
:1013A000C1916F0138E0632E600E6C2F862D0E9474
:1013B0001D0207341105B1F0F601D081CD1740F4BC
:1013C000CF5FDC1779F06C2F862D0E941D02F8CFBD
:1013D000DC1740F4DF5FCD1729F06D2F862D0E94BA
:1013E0001D02F8CF0F5F1F4F08341105C1F6209181
:1013F0006F0130917001032E000C440B550B01E07E
:1014000010E060E170E082E690E00E94C20221E01C
:1014100030E045E260E170E084E790E00E94340251
:1014200020916D0130916E01032E000C440B550B81
:1014300068E170E082E690E00E94C20221E030E0C4
:1014400045E268E170E084E790E00E94340284CED7
:1014500047EA50E069E070E089E190E00E941D03F6
:101460004AE950E064E170E089E190E073CE43E93D
:1014700050E06CE070E08CE190E00E941D038091F0
:101480007A01682D0E941C11472D481B21E030E095
:101490006CE070E08CE490E00E94340221E030E0E7
:1014A00043E76CE070E082E590E0CFCFFF920F93CE
:1014B0001F93CF93DF9361E08DE00E94C90362E048
:1014C00083E00E94C90387E090E00E94061191E04A
:1014D000811101C090E09093790188E090E00E9432
:1014E000061191E0811101C090E090937801109273
:1014F0007E0110927D011092CC011092EE010E94AB
:10150000840489E796E090933801809337018AE755
:1015100096E090933C0180933B018CE08093B8006F
:10152000C0EED0E002EF10E0FE01F4900E9431071F
:101530006F2D8FEE91E00E94EF060E94C30421966A
:101540000C171D0789F71092DC02EDEDF2E080E048
:1015500011928F5F8038E1F70E94890783E090E065
:101560000E947A0868EB7BE080E090E00E942A0409
:1015700087E58093C1028FEF0E941A08853129F018
:1015800090E080E00E947A08FFCF60E489E00E944A
:101590003F0764EF71E080E090E00E942A0460E081
:1015A00084E00E943F0760E085E00E943F0760E022
:1015B00086E00E943F076FE488E00E943F0763E0F7
:1015C00089E00E943F0767E28AE00E943F0767E1E7
:1015D0008CE00E943F0767E18DE00E943F076FE1CA
:1015E00080E10E943F078CEA97E09093030180938B
:1015F000020180916900837F846080936900E99A89
:10160000DF91CF911F910F91FF9008951F920F923C
:101610000FB60F9211242F933F938F939F93AF9305
:10162000BF938091630190916401A0916501B09195
:10163000660130915E0123E0230F2D3758F50196A6
:10164000A11DB11D20935E018093630190936401FD
:10165000A0936501B093660180915F019091600154
:10166000A0916101B09162010196A11DB11D80930D
:101670005F0190936001A0936101B0936201BF91FB
:10168000AF919F918F913F912F910F900FBE0F902F
:101690001F90189526E8230F0296A11DB11DD2CFE9
:1016A0001F920F920FB60F9211242F933F934F93D7
:1016B0005F936F937F938F939F93AF93BF93EF93BA
:1016C000FF93E0910201F09103010995FF91EF91E1
:1016D000BF91AF919F918F917F916F915F914F914A
:1016E0003F912F910F900FBE0F901F9018951F9252
:1016F0000F920FB60F9211242F933F934F935F9346
:101700006F937F938F939F93AF93BF93EF93FF93C9
:10171000E0910001F09101010995FF91EF91BF91D6
:10172000AF919F918F917F916F915F914F913F9179
:101730002F910F900FBE0F901F9018951F920F9230
:101740000FB60F9211242F933F934F935F936F9394
:101750007F938F939F93AF93BF93EF93FF9380916A
:10176000B900887F803609F44AC0F0F5883209F460
:10177000A7C018F5803109F49BC0B8F4882309F498
:10178000F9C0883009F494C0FF91EF91BF91AF91F7
:101790009F918F917F916F915F914F913F912F9189
:1017A0000F900FBE0F901F901895883109F488C0D4
:1017B000803251F78093C30114C0803409F49DC076
:1017C00040F48033B9F38833F9F68093C30185EC94
:1017D000B0C0803509F485C0883509F496C08834D6
:1017E00099F60E944208D0CF883909F48CC038F5A8
:1017F000883729F050F4883611F0803729F683E0D5
:101800008093C50110925D0157C0883809F47BC0F0
:10181000803919F0803809F0B7CF80915D018032AE
:1018200008F071C0E0915D0181E08E0F80935D0151
:101830008091BB00F0E0E35CFE4F80833DC0803BC5
:1018400039F0E0F4803A09F479C0883A09F09CCF85
:1018500084E08093C50110923A0110923901E09121
:101860003701F091380109958091390181110FC03C
:1018700081E0809339011092170109C0803C09F47E
:10188000A6CF883C09F4A3CF883B09F07DCFE09137
:101890003A0181E08E0F80933A01F0E0E95EFE4F5D
:1018A00080818093BB0090913A018091390129C0D9
:1018B0008091A0018093BB0085EC8093BC0064CF35
:1018C0009091C2018091C101981758F5E091C20131
:1018D00081E08E0F8093C201F0E0EF55FE4F8081D2
:1018E000E9CFE091C20181E08E0F8093C201809127
:1018F000BB00F0E0EF55FE4F80839091C2018091D4
:10190000C1019817C8F285E8D8CFE091C20181E003
:101910008E0F8093C2018091BB00F0E0EF55FE4F27
:1019200080838091C40181115CCF81E080939F010D
:1019300084EA8093BC001092C50126CF85EC809389
:10194000BC001092C50180915D01803230F4E091BD
:101950005D01F0E0E35CFE4F108260915D0170E09C
:10196000E0913B01F0913C018DE391E009951092EB
:101970005D010ACF1092C30134CFEFEEF1E0138284
:10198000128288EE93E0A0E0B0E084839583A68382
:10199000B78388E091E091838083EBEAF2E01082E4
:1019A000118212821382148624E130E0308B278763
:1019B0008CEE9FEF928B818B138A158A148A168680
:1019C0001586E5E9F2E010821182128213821486F4
:1019D000308B2787928B818B138A158A148A1686FF
:1019E00015861092940210928B020895CF93DF9384
:1019F000CDB7DEB728970FB6F894DEBF0FBECDBFC8
:101A0000789484B5826084BD84B5816084BD85B5D9
:101A1000826085BD85B5816085BD80916E008160E5
:101A200080936E001092810080918100826080938B
:101A3000810080918100816080938100809180008D
:101A40008160809380008091B10084608093B100B8
:101A50008091B00081608093B00080917A008460B2
:101A600080937A0080917A00826080937A008091DE
:101A70007A00816080937A0080917A0080688093F8
:101A80007A001092C1000E94560A38EEC32EDD245F
:101A9000DA94ED2CFD2C48E4242E312C86E00E94B3
:101AA0001A08898384E00E941A082981281709F4FA
:101AB00064C0821B990B97FD809626E0289FA001A9
:101AC000299F500D11245A8349838091C10291E0CE
:101AD0009093CB018093ED011092CC011092EE0116
:101AE00087E090E00E941E070E94C30469817A810A
:101AF0006132710524F080E290E09A8389836981E4
:101B0000613208F060E28091C1020E94AA05109241
:101B10007E0180937D01A981BA811A161B065CF5AE
:101B20008091DA028F5F63E00E941C11192F90935D
:101B3000DA020E949E06B4E01B9FF0011124E353D9
:101B4000FD4F61837283838394830091DA0210E0F6
:101B50000E949E06000F111F000F111FF801EF5386
:101B6000FD4F6183728383839483E981FA81369781
:101B7000FA83E983D0CF0E94C3048FB7F8942091F1
:101B800063013091640140916501509166012983A0
:101B90003A834B835C838FBF8091DB029091DA02A2
:101BA000981B97FD9D5F992309F4F5C0282F30E01D
:101BB000F901EE0FFF1FEE0FFF1FE353FD4F4181B1
:101BC0005281638174814D835E836F837887220F96
:101BD000331F220F331FF901EF53FD4F4180528015
:101BE000638074808F5F63E00E941C119093DB021E
:101BF0006D817E818F81988568387341810591055B
:101C000008F0D1C08EE480937C0062E070E080E058
:101C100090E00E942A0480917A00806480937A0088
:101C200080917A0086FDFCCF8091780080917900C8
:101C300080917A00806480937A0080917A0086FD9A
:101C4000FCCF2091780080917900382F50E040E05F
:101C500060E07CE280E090E00E94501130937C01D3
:101C600020937B01809168018823F1F00E94770323
:101C7000892BD1F48091670190E0019683709927B8
:101C800080936701682F61706093790186958170F8
:101C90008093780187E090E00E940E1160917801B6
:101CA00088E090E00E940E1110926801B0917A01D4
:101CB000BD8381E090E0B73910F084E090E00E94AD
:101CC0007A0868EC70E080E090E00E942A04ED81E0
:101CD000EF5FE0937A01E93C08F43DC00E94890778
:101CE0000E9431076EEA8FEE91E00E94EF060E949B
:101CF000C3046AE070E080E090E00E942A0460E89B
:101D000089E00E943F076AE070E080E090E00E9476
:101D10002A0480917A008F7780937A006AE070E0DD
:101D200080E090E00E942A0460E080E00E94C90305
:101D300060E082E00E94C90383B7817F846083BF33
:101D400083B7816083BF889583B78E7F83BF0E94EE
:101D5000560A10927A01809171018823E1F08091F6
:101D6000740190917501A0917601B091770129815C
:101D70003A814B815C81281B390B4A0B5B0BDA01E2
:101D8000C9014A97A105B10534F060E08DE00E94D9
:101D90009B031092710180E090E0892B09F47ECEC4
:101DA0000E9400007BCE10927A018090AB0290904E
:101DB000AC02A090AD02B090AE02C501B401A70183
:101DC00096010E9450116D817E818F819885260F2A
:101DD000371F481F591F820E931EA41EB51EC50132
:101DE000B401A70196010E9450118D819E81820F3E
:101DF000931F9E838D83809179018092AB02909294
:101E0000AC02A092AD02B092AE028111BAC1809034
:101E1000950290909602A0909702B0909802C5010A
:101E2000B401A70196010E945011240D351D461DD5
:101E3000571DCA01B901680D791D8A1D9B1D60934C
:101E40009502709396028093970290939802A7014F
:101E500096010E945011420E531EB20189E992E090
:101E60000E94B007BC0185E992E00E94D407B82E19
:101E70006D817E818FEA92E00E94B007BC018BEAFF
:101E800092E00E94D407382F40917801442309F44E
:101E9000B5C1AA27BB27A419B509BE83AD836D813F
:101EA0007E8177FF04C0695F7F4F7E836D838D8164
:101EB0009E81F3E095958795FA95E1F79E838D8352
:101EC00080918B0290E0FC01E550FE4FAD81BE8118
:101ED000A058BF4FBE83AD83B7FF02C01E821D82D4
:101EE0006D817E816F3F710529F024F0AFEFB0E086
:101EF000BE83AD83BD81B0830196B1010E943C11C8
:101F000080938B0241113B2D332309F4B3C08091A0
:101F1000740190917501A0917601B09177012981AA
:101F20003A814B815C81281B390B4A0B5B0B60E6C5
:101F30007AEE80E090E00E945011DA01C901019729
:101F4000A109B109873C9105A105B10548F4B90182
:101F50008CE892E00E94B007909373018093720125
:101F600029813A814B815C81209374013093750102
:101F7000409376015093770161E08DE00E949B03CE
:101F800081E0809371011091A2023091A3023D8300
:101F90004090AB025090AC026090AD027090AE02E7
:101FA00060919502709196028091970290919802AB
:101FB00028E130E040E050E00E945011A091B802CA
:101FC000B091B902B7FD1396B595A795B595A795AC
:101FD0000E947A1120E031E040E050E00E94501170
:101FE00049015A0127EE33E0181419041A041B049E
:101FF0002CF5812F9D8197FD0396AC015595479552
:10200000559547955E834D83C301B20128E130E0C9
:1020100040E050E00E945011AD81BE810E947A11D3
:1020200020E031E040E050E00E945011A4E6B0E032
:102030000E946F11A50194010E9450114FEE4203BE
:10204000C001439F900D11248E52974D64E670E0BD
:102050000E943C117093700160936F01283B310521
:1020600048F42A5F3E4FF901249130E030936E012D
:1020700020936D018091690190916A01A0916B019B
:10208000B0916C0129813A814B815C81281B390B0D
:102090004A0B5B0BDA01C901C397A105B1050CF42A
:1020A0005BC049815A816B817C8140936901509367
:1020B0006A0160936B0170936C01EBEFF1E05FEFED
:1020C0005D8320E08191281708F4282F6D81861701
:1020D00008F48D8383E492E08E179F0799F7FD81C2
:1020E000EF2FF0E0FE83ED8330E02E1B3F0B37FF38
:1020F00002C02D5F3F4F35952795359527952F5F6A
:1021000080918B0203E412E030E04FE1E82FF0E031
:10211000DF01A550BE4F8C9190E06D817E81861BC2
:10212000970B53E0880F991F5A95E1F7B9010E9468
:102130002811842F861BD8018D938D01CF01019624
:10214000B1010E943C11EBE8F2E0E017F107F1F673
:1021500082E090E00E947A0880916801882371F003
:102160000E947703892B51F485E090E00E947A0861
:102170006CE474E080E090E00E942A041092680110
:10218000EACD6D817E818FEA92E00E94B0079E8346
:102190008D838090950290909602A0909702B090C7
:1021A0009802C501B401A70196010E945011240DA7
:1021B000351D461D571DCA01B901680D791D8A1DBF
:1021C0009B1D609395027093960280939702909363
:1021D0009802A70196010E945011B201620F731F6D
:1021E00089E992E00E94B0072C01BC0185E992E0E8
:1021F0000E94D407B82E6D817E8141CEED81FE8193
:10220000F195E195F109FE83ED8349CEF999FECF71
:1022100092BD81BDF89A992780B50895262FF99926
:10222000FECF1FBA92BD81BD20BD0FB6F894FA9AB9
:10223000F99A0FBE01960895991B79E004C0991F81
:10224000961708F0961B881F7A95C9F78095089510
:10225000AA1BBB1B51E107C0AA1FBB1FA617B707CC
:1022600010F0A61BB70B881F991F5A95A9F78095E8
:102270009095BC01CD01089597FB072E16F40094AC
:1022800007D077FD09D00E94281107FC05D03EF445
:10229000909581959F4F0895709561957F4F089512
:1022A000052E97FB1EF400940E94671157FD07D07E
:1022B0000E94821107FC03D04EF40C9467115095D4
:1022C0004095309521953F4F4F4F5F4F0895909522
:1022D0008095709561957F4F8F4F9F4F08950E9415
:1022E000AA11A59F900DB49F900DA49F800D911DE4
:1022F00011240895B7FF0C946F110E946F11821B77
:10230000930B0895A1E21A2EAA1BBB1BFD010DC061
:10231000AA1FBB1FEE1FFF1FA217B307E407F50795
:1023200020F0A21BB30BE40BF50B661F771F881F71
:10233000991F1A9469F760957095809590959B0107
:10234000AC01BD01CF010895EE0FFF1F0590F49180
:10235000E02D0994A29FB001B39FC001A39F700D0F
:10236000811D1124911DB29F700D811D1124911D9D
:102370000895F894FFCF5C045C0400000000EF06B1
:0C238000C206A9077B06BB068B067C0684
:107E0000112484B714BE81FFF0D085E080938100F7
:107E100082E08093C00088E18093C10086E0809377
:107E2000C20080E18093C4008EE0C9D0259A86E02C
:107E300020E33CEF91E0309385002093840096BBD3
:107E4000B09BFECF1D9AA8958150A9F7CC24DD24C4
:107E500088248394B5E0AB2EA1E19A2EF3E0BF2EE7
:107E6000A2D0813461F49FD0082FAFD0023811F036
:107E7000013811F484E001C083E08DD089C08234E0
:107E800011F484E103C0853419F485E0A6D080C0E4
:107E9000853579F488D0E82EFF2485D0082F10E0AE
:107EA000102F00270E291F29000F111F8ED06801E7
:107EB0006FC0863521F484E090D080E0DECF843638
:107EC00009F040C070D06FD0082F6DD080E0C81688
:107ED00080E7D80618F4F601B7BEE895C0E0D1E017
:107EE00062D089930C17E1F7F0E0CF16F0E7DF06D8
:107EF00018F0F601B7BEE89568D007B600FCFDCFD4
:107F0000A601A0E0B1E02C9130E011968C91119780
:107F100090E0982F8827822B932B1296FA010C0160
:107F200087BEE89511244E5F5F4FF1E0A038BF0790
:107F300051F7F601A7BEE89507B600FCFDCF97BE46
:107F4000E89526C08437B1F42ED02DD0F82E2BD052
:107F50003CD0F601EF2C8F010F5F1F4F84911BD097
:107F6000EA94F801C1F70894C11CD11CFA94CF0C13
:107F7000D11C0EC0853739F428D08EE10CD085E9AC
:107F80000AD08FE07ACF813511F488E018D01DD067
:107F900080E101D065CF982F8091C00085FFFCCF94
:107FA0009093C60008958091C00087FFFCCF809118
:107FB000C00084FD01C0A8958091C6000895E0E648
:107FC000F0E098E1908380830895EDDF803219F02E
:107FD00088E0F5DFFFCF84E1DECF1F93182FE3DFCA
:107FE0001150E9F7F2DF1F91089580E0E8DFEE27F6
:047FF000FF270994CA
:027FFE00040479
:00000001FF
